:1000000012C01895189518951895189564C01895EC
:100010001895189518951895189518951895189578
:100020001895189518958FED8DBFC0ECE8EB4E2E06
:10003000DD275D2EEEE7F0E0A0E6B0E0A89584B7FE
:10004000082E877F84BF88E1992781BD91BD8827CD
:100050008D933197E9F73AD266248FEF87BB8FEF04
:1000600088BB87EC81BB8FEF82BB1CD28CE076D241
:1000700084E083BF80E080BF89B7826089BF84B796
:10008000877F84BF8FE181BD87E081BD789480E95F
:1000900091E0ABE68D939C9381B5886081BDA2E62B
:1000A0008C9186FB0EF007C0809162008F7B80935D
:1000B000620012D141D1A2E68C9187FB0EF008C0FC
:1000C000809162008F7780936200A89560D0AED057
:1000D000E6CFF894FFCF0F921F922F923F924F924C
:1000E0005F927F92AF92BF920F931F932F933F9394
:1000F0004F935F936F937F938F939F93AF93BF9330
:10010000CF93DF93EF93FF938FB78F9383E8809321
:100110005200A0E68C918F5F8C93009160000931B2
:1001200009F019C080E080936000809162008064D3
:1001300080936200A1E68C918F5F8C9300916100A7
:100140000A3009F008C080E080936100809162006D
:100150008068809362008F918FBFFF91EF91DF9154
:10016000CF91BF91AF919F918F917F916F915F914F
:100170004F913F912F911F910F91BF90AF907F9022
:100180005F904F903F902F901F900F901895A2E690
:100190008C9185FB882780F9809580FBA2E68C9165
:1001A00085F98C93F89482E0E0E339D2A2E68C9151
:1001B00085FB0EF011C06CEC82E0E0E3BB27A6E10A
:1001C00021E02A9358D264E482E0E0E3BB27A6E171
:1001D00021E02A9350D228C06CEC82E0E0E3BB27F8
:1001E000A6E121E02A9347D26EEB82E0E0E3BB2751
:1001F000A6E121E02A933FD282E0A9E6E0E322E0F3
:100200002A9373D2A9E60D911C914AE050E029D1BE
:10021000A9E60D931C93A9E60D911C9140E150E0D5
:1002200006D1A9E64D935C9378940895ABE60D91C1
:100230001C91A9E64D915C91041B150BADE60D9345
:100240001C93ADE60D911C9147E050E0040F151F83
:10025000ADE60D931C93ADE60D911C91003050E07E
:10026000150714F009F004C080E0809370000EC000
:1002700080916D008093700000917000023310F047
:1002800009F001C003C082E380937000AFE68C9157
:100290008F5F8C9300916F00023309F003C080E000
:1002A00080936F004091700000916F00041708F078
:1002B00002C0969801C0969AA9E60D911C91083546
:1002C00052E0150708F406C0969A82B391E0892798
:1002D00082BB01C0909A0895A0E30C9103FB81E0DA
:1002E0000EF480E08F93ABE60D911C91083552E03F
:1002F000150781E010F009F080E09F9189238823A1
:1003000009F402C0ABE660D0A0E30C9104FB81E0ED
:100310000EF480E08F93ABE60D911C910A3F50E004
:10032000150781E008F480E09F918923882309F470
:1003300002C0ABE650D008958FE711E0C2D0A9E625
:100340008D919C91A7E68D939C931CD08FEB11E02F
:10035000B8D0ABE68D919C91A7E68D939C9312D07B
:100360008FEB17E0AED0009170000A3008F003C0A8
:10037000ECEFF7E091D0A0EAB0E0E0E7F0E0F4D1F4
:1003800083D00895A7E60D911C914AE050E04FD02C
:10039000A4E64D935C93A0EAB0E0E4E6F0E0D5D1AA
:1003A00073D0EEEFF7E078D0A7E60D911C914AE00C
:1003B00050E03DD0A4E60D931C93A0EAB0E0E4E643
:1003C000F0E0C3D161D00895ED91FC91EF5FFF4F54
:1003D000FC93EE930895ED91FC91E150F040FC9375
:1003E000EE93089508D03DD000FC10D0089503D0BE
:1003F0001ED001F8F9CF0024E89457FF02C009D0BD
:10040000689400F80BD010F80124089502D009D0A8
:100410000895509540954F5F5F4F0895E89417FFFA
:100420000895009510950F5F1F4F68940895352F1C
:10043000242FE894452B11F468940895512F402FF0
:100440000027112780E1440F551F001F111F021BB9
:10045000130B416018F4020F131F4E7F8A9599F712
:100460000895752F642F55274427FF93F1E1889451
:1004700005C010F4460F571F5695479517950795D9
:10048000FA95B9F7FF910895A0EAB0E08D9188231D
:1004900011F05ED0FBCF08959CD0802D11F058D084
:1004A000FBCF089581E05AD00ED080E857C08FE787
:1004B000213039F08FEB223021F08FE8233009F022
:1004C0008FEC810F4BC083E0992774C08AEF90E0D6
:1004D00071D0BA9ABB9ABD9ABC9ABF9ABE9AC69876
:1004E00085E090E067D0C798C298C398C59AC49A2F
:1004F000C79AEF93FF93E4ECF0E050D0FF91EF91B7
:10050000C79855D0C79AEF93FF93E4ECF0E046D03C
:10051000FF91EF91C7984BD0C79AEF93FF93E4EC0C
:10052000F0E03CD0FF91EF91C79841D0C498C79AB2
:10053000EF93FF93E4ECF0E031D0FF91EF91C79897
:1005400036D088E20BD08EE009D086E007D008953F
:10055000C69A829505D004D02AD00895C698F9CFBE
:10056000859510F4C49A01C0C498859510F4C59A75
:1005700001C0C598859510F4C39A01C0C3988595AC
:1005800010F4C29A01C0C298C79AEF93FF93E4ECAB
:10059000F0E004D0FF91EF91C79808953197F1F7FB
:1005A0000895689462F80895E89462F8089581E0E7
:1005B00090E000C0EF93FF93EE27E82BE92B31F09A
:1005C000E0EDF7E03197F1F70197D1F7FF91EF9167
:1005D0000895C89531960020089591E0882321F070
:1005E0008894991F8A95E9F7892F9095089501813C
:1005F000082B0183128119231283000000000000E0
:1006000000000000000000000000000000000000EA
:100610000000000000000000000000000895C1DF9D
:10062000FF27DBDFE4DFEF93FF93ECEBF3E0B6DFD4
:10063000FF91EF91182B128309230183EF93FF930E
:10064000E0EBF0E0ABDFFF91EF911081182359F45C
:10065000EF93FF93ECEBF3E0A1DFFF91EF911081BB
:10066000182309F0A1DFEF93FF93ECEBF3E096DFA3
:10067000FF91EF910895B1DFFF2729915D9148E047
:10068000B6DF0000000000000000000000000000D5
:10069000000000000000000000000000000000005A
:1006A00000000000579510F4182B1283EF93FF936E
:1006B000E4E7F0E073DFFF91EF91182B1283000065
:1006C000000000000000000000000000000000002A
:1006D000000000000000000000000000000000001A
:1006E0004A9571F62A9551F6089577DFFF272991EB
:1006F00048E055277CDF09230183EF93FF93E8E06F
:10070000F0E04CDFFF91EF9188941081182309F0FD
:1007100008945795EF93FF93E6E5F0E03FDFFF91F4
:10072000EF914A9539F75D932A9511F70895000FD7
:10073000111F221F331F08950095109520953095A5
:100740000F5F1F4F2F4F3F4F0895019110810EC033
:1007500001911191219130810BC00191108117FFFE
:1007600005C03FEF2FEF04C0008111272227332758
:1007700037FF03C0E1DF8DE28D93CF93DF93CF92FC
:10078000DF92EF92AA24BB24CC24DD24EE2440E2A5
:10079000CAE0DD2755E093E38881890F87FD9F70CC
:1007A00083FD907F891B89935A95A9F7C0DFAA1C06
:1007B000BB1CCC1CDD1CEE1C4A9551F7E894EFE005
:1007C000FF2782910ED0EB30E0F71EF068948A2D5F
:1007D0000CD088278D93EF90DF90CF90DF91CF9151
:1007E0000895982F829501D0892F8F70805D26F013
:1007F000803309F4089568948D93089520002E00A5
:00000001FF
